:020000020000FC
:1000000070CD0000000000001FC0A5C193C000001B
:1000100000009DC000000000000000000203040674
:10002000080C10182030406080000406080C1018DE
:100030002030406080A0C00000070F1F3F00050572
:100040000D050305030302004FB662FD0EC05520E7
:1000500009F00994C52DC095089483FDC795C4BDCA
:10006000C093A10064604FBE1895C09164000894CD
:1000700083FDC795C4BDC093A1006B7FC091640090
:10008000CF3F09F420C070FF02C082FD05C04FBE03
:10009000939894989598189575FD0EC065FD0CC0C1
:1000A000C091B300C0FD9298C1FDC298C2FDC19835
:1000B000CAEFC095CA95F1F79398949895982092B5
:1000C000A1004FBE189524BCCC27C064C8BF646093
:1000D000F6CFC0CF70FFBECF65FDBCCF939ABACF2D
:1000E00070FFB8CF65FDB6CF949AB4CF70FFB2CF92
:1000F00065FDB0CF959AAECF929A70FFABCF65FDFC
:10010000A9CFC7E0CA95F1F7939AA4CFC29A70FF1E
:10011000A1CF65FD9FCFC7E0CA95F1F7949A9ACF1A
:10012000C19A70FF97CF65FD95CFC7E0CA95F1F7EB
:10013000959A90CF4FB6C9B7CF7EC9BF6E7FCCB569
:10014000CE0DDDB5DF1DDBBDCABD4FBE18953FB678
:100150008F7EA9B7A072A2118061A9B7AF7DA9BF98
:10016000A9B7AE7FA9BF7894A0916800AA2341F0F7
:1001700085FD2BC0A0916800AA95A093680025C0BA
:1001800040E050E085FD15C0A6B396FDA095A0FD0A
:100190004FEFAEB5A06496FDAF7BAEBDAA27A062BF
:1001A000A8BF8D7FA6B396FDA095A0FD5FEF451774
:1001B00039F7A8E161FDA093680085FD03C0A8E1BF
:1001C000A093680040939700816085FD0EC0A091C8
:1001D0006900AA2331F0A0916900AA95A093690053
:1001E00004C08061AA27A062A8BF80FF38C0A09188
:1001F00097004A2F61FF8E7F85FD18C0403F08F0B1
:1002000040EFA42FA295AF704A0F5091B800533021
:1002100069F0A695A69550FD01C0A69552FD03C0B4
:10022000A41B4A2F03C04A0F08F44FEFA091A0006F
:100230004A1708F44A2F40936100A72FA67079F05F
:10024000A0916D00A695A69556E0A50F509161006E
:10025000A50FA093610018F4AFEFA0936100A091E7
:100260006100A093630040916300A0919C004A1735
:1002700008F04A2F542EA091A200AA2309F422C00C
:10028000542F5A1B10F4A42F50E0BA2E8894AA1FA2
:10029000AA2EA091A400A095AA22A50E58F0A09184
:1002A000A300A21509F0AA95AA0EA093A30048F0F6
:1002B0004A2D08C0A091A300BA1608F0A395A093F8
:1002C000A3004FEF409364007F7D485F08F07062A9
:1002D000A52DA03408F06860A0916000A395A093BC
:1002E000600059F0F894A9B7A160A9BF84FF03C0CA
:1002F000A9B7A062A9BF3FBE1895A0917400A395AD
:10030000A093740041E050916800552329F085FFC7
:1003100003C05A9550936800A0919700A13018F03F
:1003200020929A000DC020929B002092A500A091DF
:100330009A00AF5FA0939A0018F0AFEFA0939A00D5
:10034000F894A9B7A160A9BF84FF03C0A9B7A062B0
:10035000A9BF3FBE18953FB646B557B58F7EA9B722
:10036000A072A2118061A9B7AF7DA9BFA9B7AE7F66
:10037000A9BF789481FD25C0AEB5AF7B96FDA06482
:10038000AEBD8260A6B396FDA095A0FF05C04093C8
:100390006500509366003FC1AEB5A06496FDAF7B8B
:1003A000AEBDAA27A062A8BF8D7F85FF01C026C170
:1003B00040E0A6B396FDA095A0FD20C14093970014
:1003C0000FC1AEB5A06496FDAF7BAEBD8D7F61FF62
:1003D00072C0AEB5AF7B96FDA064AEBDAA27A06289
:1003E000A8BF82604093920050939300A090900029
:1003F0004A19B09091005B09BB24A22C4C385205DD
:1004000018F42092960049C0A091D600AA2359F171
:10041000483C520528F4A0E1BA2EAAE0AA2E23C037
:100420004836A1E05A0728F4A8E0BA2EAFE0AA2E79
:100430001AC0403DA2E05A0728F4A4E0BA2EAEE16B
:10044000AA2E11C0403AA5E05A0728F4A2E0BA2E1D
:10045000ACE3AA2E08C04839A8E05A0720F4A1E06E
:10046000BA2EA8E7AA2EC42EA0919400CA1AD52E9F
:10047000A0919500DA0ADD202AF4AFEFC094D09461
:10048000CA1ADA0A20929600A8E0A210A0E0CA14C4
:10049000DA0618F4A1E0A0939600409394005093DC
:1004A000950040919200509193004093900050939A
:1004B000910002E095C0A09165004A1BA0916600E2
:1004C0005A0B94FD80C093FD7EC092FD7AC086FFDA
:1004D00003C0D52EC42E0CC05695479591FD71C012
:1004E0005695479590FD6DC0D52EC42ED694C794D1
:1004F00061FD17C0AC2DAC51AD2DA24008F005C078
:10050000DD2079F4AC2DA85C60F4A0916700A39580
:10051000A0936700AA3008F471C020929700816010
:100520006DC0A0916700AA2319F0AA95A093670057
:10053000A22C5091BC0097FD06C0A090CA00533079
:1005400011F4A090D200AAEFAA0EA22DA21DCA18E3
:10055000DA0A4FB74170533049F4442321F087FD44
:1005600005C0806803C087FF01C08F77442359F01E
:10057000533031F4AFEFC094D094CA1ADA0A03C0F2
:1005800040E050E020C0533049F4CC0CDD1CAAE020
:10059000CA1AD20818F4A0E0CA2ED22CAFEFCA169D
:1005A000D20418F04FEF50E00EC0A091AE00CA9EEA
:1005B000412D000C441F50E008F012C04FEF50E0F6
:1005C0000FC05695479594FF07C0552309F04FEF8C
:1005D000A42FA6954A0F521D4F3F520508F04FEF2A
:1005E00040939700816061FF09C0AFE1A095A92306
:1005F000AB299A2F8F7DBB2009F48062A8E1A093DC
:10060000680085FF03C0AAE0A093680061FD03C0F5
:1006100085FD01C08F7E85FD03C0A6E0A093690023
:10062000F894A9B7A160A9BF84FF03C0A9B7A062CD
:10063000A9BF3FBE189511E00AC013E008C01AE038
:1006400006C01EE104C014E602C018EC00C005E1BB
:10065000BB27BA95F1F70A95D9F71A95C1F708950E
:100660002AE338E709C020E33CE806C02AE234EB7D
:1006700003C025E238EC00C012E095FD9F7D95FF98
:100680009062BB27C29ABA95F1F7949ABA95F1F79E
:100690009498BA95F1F7C298BA95F1F7939AB091F8
:1006A000AF00BA95F1F79398B7E8BA95F1F71A95B4
:1006B00021F7022FB22FBA95F1F70A95D9F73A959B
:1006C000D9F6C29A0895221B39E0001F3A9509F421
:1006D0000895221F211B18F4210F8894F6CF089447
:1006E000F4CF622C722CB0E08894B395221F331F94
:1006F000E0F7379527958894912E802E020B130BE7
:1007000010F4192D082D10F4889401C00894661C6B
:10071000771CBA9571F7172D062D0895322D1123E8
:100720002AF43A9500951095031B130BF894029F39
:10073000712C002D129F912C802C7894780C172D01
:10074000921C292DB4E06B2E2695179507956A9477
:10075000D9F7332321F000951095031B130B08954F
:10076000089510917B00169500917A000795B0913D
:100770007F00B01B0B2FB0918000B10B1B2F28F412
:100780000038BFEF1B0740F009C00F37120508F40F
:1007900005C00FE710E002C000E81FEF00938400DF
:1007A00010938500089500918400B09181000B0F93
:1007B00010918500B09182001B1F20E030918500D0
:1007C00033230AF42A95B09183002B1F1AF4203F9B
:1007D00040F00AC02F3008F407C00FEF1FEF2FE0E2
:1007E00003C000E010E020EF30916300B0919C0066
:1007F0003B1718F4323030F009C0B0918500BB23AC
:100800005AF004C0B0918500BB2332F400938100FC
:10081000109382002093830008952091D8000091C6
:100820008400000F10918500111F78DF11232AF436
:100830000038BFEF1B0740F009C00F37120508F45E
:1008400005C00FE710E002C000E81FEF002352F0E0
:10085000B0916200B01B0B2F18F0013008F00AC0F5
:1008600001E008C000950F5FB09162000B0F08F027
:1008700001C00FEF0093860008952091D9000091E8
:100880008200109183004ADF11232AF40130BFEF68
:100890001B0740F009C00F3F120508F405C00FEF19
:1008A00010E002C001E01FEF112352F0B09186006A
:1008B000B01B0B2F18F0013008F00AC001E008C08F
:1008C00000950F5FB09186000B0F08F001C00FEF8D
:1008D0000093630008950FEF677F71FD29C072FDDB
:1008E00009C06860B0917B00BA3020F0B52DB034FB
:1008F00008F4677FB091D500BB23D1F0B0917B00A5
:10090000BB23B1F00FEF10917B00DDDEF894B091C6
:10091000730072FDB5E00B9F112D002D789411230B
:1009200009F00FEFB0919F000B1710F400919F009A
:1009300000939E00089500917A0010917B0000546E
:100940001140B0919E0010F4BA9501C0B39511F01A
:10095000B0939E00089500C008952091B700B6B1ED
:10096000B6FDFBCF04B115B1B6B1BF77B6B9B09142
:10097000AC00B395B093AC00B83060F12092AC00FD
:10098000B091D400BB2321F1112329F0B091AD0027
:10099000BF3F61F009C0B091AD000B1739F020F4F2
:1009A000BB2321F0BA9502C0B395E1F300919C00FE
:1009B000B093AD00B93B50F400ECBA3A38F400E81B
:1009C000BB3920F400E4BC3808F400E000939C003C
:1009D000777F0895B0919C00B39511F0B0939C007F
:1009E000B091AC00B73009F47860089502E3F89450
:1009F000B091DA000B9F012D000C001F7894B0918C
:100A00009C000B1710F000919C0000936100009374
:100A10006300502E0093640000939F00089520927D
:100A20007A00B0EFB0937B000895F8940CB51DB533
:100A30002091740078943091750060907600009356
:100A4000750010937600031B160971FD03C076FD37
:100A500081C02BC070907700209377002709222354
:100A600011F00FEF1FEF8090780090907900309395
:100A70007800609279006918161910937C00009133
:100A80007500109176000819190920917A003091AB
:100A90007B0036952795020F131F10F40FEF1FEF01
:100AA00000937A0010937B0029C020917A00309146
:100AB0007B003901B4E08B2EB2E09B2E343010F075
:100AC0008A949A94383010F08A949A947694679421
:100AD0008A94E1F726193709992021F01695079590
:100AE0009A94E1F7200F311F20937A0030937B0016
:100AF00028F43FEF30937A0030937B00323008F4D3
:100B0000706471FF02C0B3E00DC0B091C6000091E7
:100B10007100023838F0B395003A08F0B395B6305A
:100B200008F0B5E09B2EB4E08B2E10917B00009175
:100B30007A0024E0169507952A95E1F7081912091D
:100B400028F0B02FB250B12FB20910F402E010E03B
:100B5000980126C020917A0030917B00390176946B
:100B600067946694669466942619320906950695EC
:100B7000200F321D20937A0030937B00323008F032
:100B80007F7B04E036952795369527952695269503
:100B9000201B10F0223008F422E089019090C6005A
:100BA00060FDFECFE0908C00F0908D006160B9B7E1
:100BB000B061B9BF380176FD44C076946794009364
:100BC0008C0010938D00B92DB330E1F0B0FD04C05E
:100BD000060D171D930106C0000F111F02501209C8
:100BE00022E030E0B92DB33068F020938E003093CE
:100BF0008F00009388001093890060928A007092A1
:100C00008B003DC000938E0010938F0020938800CE
:100C10003093890060928A0070928B0071FF10C03F
:100C2000B0916D00B33060F000918F0010917C00A6
:100C30001595010F28F022F020928E0000938F006E
:100C40001EC0669400938C00B92DB33091F0B0FDB6
:100C500003C0060D262D03C0000F025022E0B92D5F
:100C6000B33038F020938E000093880060928A00A1
:100C700006C000938E002093880060928A00009145
:100C80007D0002FD0350013049F495FD12C0B0B75C
:100C9000B860B0BFB0E0B06CB7B90EC0023039F484
:100CA000B0B7B860B0BFB1E0B06CB7B905C095FDE2
:100CB000EECFB0B7B77FB0BF0091A400000F10F423
:100CC000BBE60B270093A40060FDFECFB2E0B0931B
:100CD0006E006160B9B7B061B9BFB72FB670A1F04F
:100CE00020917A0030917B0036952795F8940CB5C9
:100CF0001DB5020F131F1BBD0ABD6160B0E1B8BF77
:100D0000B9B7B061B9BF78940895606120927E0050
:100D100020E067FD20E206C0606120927E0020E2B4
:100D200067FD20E0789401E076FD11C0B72FB67022
:100D300009F06F7EB0917B00B55048F002E0B550ED
:100D400020F003E0B55008F006E071FD0AE060FD18
:100D500012C0B0917E00BB2371F071FF08C0B0914A
:100D60006D00B33020F0B0916E00BA9519F478940C
:100D700070615EC0AEDF789400000000F89476FDEC
:100D800016C010917B00173008F017E0B5E01B0F7C
:100D900072FD10E183FF110F62FF110F71FD12E868
:100DA000B4B56090A100B61990F2B10B80F2B0B763
:100DB0001B2FB77FB0BFB8B1B0B713FDB860B0BFDD
:100DC000B0917E00B395B0937E00B8B176FD06C0B9
:100DD000B1E071FDB2E0BA95F1F7B8B1B072B217F7
:100DE00009F01BC071FF05C003950A3008F0039598
:100DF000AECF64FF97CF6F7E3CB56DB470907A0034
:100E000080907B00370D681C6BBC3ABD6160B0E11F
:100E1000B8BFB9B7B061B9BF85CFB0916D00B2307E
:100E200008F480CF64FD7ECF0A9509F090CF7F7ED5
:100E300020918E0030918F00F894B0E1B8BF0CB5CE
:100E40001DB5020F131F1BBD0ABDE0908800F09076
:100E500089006160B9B7B061B9BF7894B72FB67037
:100E600039F0B0916D0072FFB395B0936D0009C079
:100E700074FF07C067FD05C064FD03C0BF91BF914B
:100E8000ECC4089500E063FF03C064FF01C001E00B
:100E9000F89410917100B7E01B9F212D102D7894CC
:100EA000200F26951795269517952695179510933B
:100EB0007100183718F4B8E7B09371000091710011
:100EC000B09172000B1720F06062939894989598F7
:100ED00060FDFECFE0908A00F0908B006160B9B7B2
:100EE000B061B9BF0895AC98B2E095FD07C0F89421
:100EF000B0937D00C29A92987894EAC0F894B09327
:100F00007D00C29AC1987894E3C0AC9AB3E082FFA6
:100F100024C095FD11C002E0F894B0937D00E6E88E
:100F2000F0E00093B3009598C19A62FF02C0949AD2
:100F300001C0C2987894CCC002E0F894B0937D00D0
:100F4000E6E8F0E00093B3009398929A62FF02C043
:100F5000949A01C0C2987894BBC095FD0BC0F894D8
:100F6000B0937D00E0E7F0E0959862FF01C0949AAD
:100F70007894AEC0F894B0937D00E0E7F0E09398E9
:100F800062FF01C0949A7894A3C0AC98B4E095FD38
:100F900007C0F894B0937D00929AC198789498C055
:100FA000F894B0937D00C19A9298789491C0AC9ACD
:100FB000B5E082FF24C095FD11C001E0F894B09324
:100FC0007D00ECE7F0E00093B3009498C29A62FFD2
:100FD00002C0939A01C0929878947AC004E0F89481
:100FE000B0937D00E0E9F0E00093B3009498C29ADA
:100FF00062FF02C0959A01C0C198789469C095FDBE
:101000000BC0F894B0937D00EAE6F0E0949862FF9C
:1010100001C0939A78945CC0F894B0937D00E6E7A1
:10102000F0E0949862FF01C0959A789451C0AC9812
:10103000B6E095FD07C0F894B0937D00C19AC298C0
:10104000789446C0F894B0937D00929AC2987894B0
:101050003FC0AC9AB1E082FF24C095FD11C004E00E
:10106000F894B0937D00E0E9F0E00093B30093982A
:10107000929A62FF02C0959A01C0C198789428C0E4
:1010800001E0F894B0937D00ECE7F0E00093B3004A
:101090009598C19A62FF02C0939A01C09298789481
:1010A00017C095FD0BC0F894B0937D00E6E7F0E023
:1010B000939862FF01C0959A78940AC0F894B0930F
:1010C0007D00EAE6F0E0959862FF01C0939A78947B
:1010D0006F7D089529E630E0F9012092B3009398DE
:1010E00094989598929AC29AC19A6B7F0895A4EBAE
:1010F000B0E00FEF0D930D930D930D9303E00D935F
:1011000004E00D930AE00D9303E00D9301E00D93CD
:1011100001E00D93A0ECB0E001E00D930FEF0D9313
:101120000D930D930D930D9303E00D930FEF0D931E
:101130000FEF0D930D9305E20D9300ED0D930AEF64
:101140000D930AEF0D9304E00D930FEF0D9301E063
:101150000D9300E00D930AE70D930FEF0D9300E060
:101160000D9301E00D9300E00D9303E00D930895BE
:101170002091BB008B7F233009F48460B091BC00C8
:10118000B33019F09F7DB1FD90629F7BB091BD009F
:10119000B1FD9064223011F0886001C0877F08950E
:1011A0000A95E00FF21DB4910895ECE1F0E0009192
:1011B000B400F6DFB093D800ECE1F0E00091B500A8
:1011C000EFDFB093D900EAE2F0E00091BA00E8DF87
:1011D000B093DA00B091D0000FEF1CE0B23011F400
:1011E00000EA1AE0B33011F402E815E0009372004F
:1011F00010937300E8E3F0E00091D700D1DFB093E3
:10120000A200089508952091CA003091CB00B091BA
:10121000BC00B33009F43E5097FF02C020E03FEF1E
:10122000B32FB21B6B2EB25810F4B2E86B2E00E055
:101230000395609EB12DBD57D8F30093AE0008957D
:101240009068E1DFFED920E030E0B0E16B2EF5D907
:10125000B09197002B0F321D6A94C9F7B4E0369510
:101260002795BA95E1F7822E9F77CDDF0895F89400
:10127000E3E0F0E0B9E0B7BFB491B078C1F3F8941F
:10128000A895B1B5B861B1BDB0E0B1BDB4E0BEBF25
:10129000BFE5BDBF1FDFB6E0B8BBB6E1B7BBB8E086
:1012A000B5BBBCE1B4BBB4E0B2BBBCE3B1BB222470
:1012B000A0E0B0E02D92AA31E9F7A0E6B0E00FEF90
:1012C0002D920A95E9F7B1E0B093A40010DFF9D2AE
:1012D000B7E0B06CB7B9B6B1B460B068B6B9009158
:1012E000CC000093AF00B1E0B0936A00F894ADD9A0
:1012F000B7D9A7D9B8D9A5D9B9D9A3D969D3A5D907
:10130000A4D9A1D9F8940AEF1AEFA6B396FDA09537
:10131000A0FF1FC01A95C9F70A95B1F7E0E0FCE1FC
:10132000B591B43E39F4B591B03E21F4B591BF3FCB
:1013300009F40CC0E0E0F395F395B591B83F49F49A
:10134000B591B43931F4B591BA3A19F4EE27F6955E
:1013500009940EDF2ADF56DF56DF0091CC000093A0
:10136000AF00B8DEB2E0B3BFB2E0BEBDB2E0B5BD23
:10137000B1E5B8BFB9BFB0B70B2FB77FB0BFB8B139
:10138000B0B703FDB860B0BF56D97894E4DABEB503
:10139000B06496FDBF7BBEBDB9B7B062B9BFBB2715
:1013A000B062B8BF8D7F51D9626033E02CE0B0915C
:1013B0009600BB2321F42CE03A9509F4A3CF41D940
:1013C00080FFA0CF8E7FB0919700B23078F3B92F15
:1013D000BF710091990000939800B0939900B017E5
:1013E00029F72A9521F76D7FBEB5B06496FDBF7BC6
:1013F000BEBDBB27B062B8BF8D7FB091D600BB2306
:1014000021F48062B92FB0709B2F8F7B20926700F0
:101410001AD985FF05C0B0916700BA3008F0806422
:101420000CD902E085FF01C000E0B0919700B01731
:10143000B8F3F89415D914D913D9789406D9209211
:101440008700B091BC00B33009F474C0F6D8B091F5
:10145000C000B13008F46EC0B0916A00B13008F439
:1014600069C085FD18C0B0919700BF3F08F462C005
:10147000F894FFD87894E7D8B0919700B130C0F7CE
:10148000F894EED8DCD8ECD87894DDD8B0919700F9
:10149000BF3FB0F3CFC2B8E09B2E9068F894B3DEA4
:1014A0007894D1D8F8949F77AEDE80909700B09171
:1014B0009700BF37789408F445C0BDD8F894D9D8C0
:1014C00078949A9451F7BCDEB82DB550B093CB0008
:1014D000BCD8F89423D281D27894BAE09B2E90683D
:1014E000F89491DE7894AFD8F8949F778CDE809052
:1014F0009700B0919700BF37789478F79CD8F8940C
:10150000AFD89DD8ADD878949A9449F799DEB82D84
:10151000BB5FB093CA0099D8F89400D26DD278948A
:1015200092D8F89470DE7894B0919700BF3F08F499
:1015300098CF80C200919700B09187000B1710F0F0
:101540000093870080D801E0B091BC00B35009F44B
:1015500005E0B0919700B01708F073CFF89489D8E0
:1015600088D887D8789471D820926A0020926B002E
:1015700020926C00B0916B00B395B0936B00BF3FAD
:1015800069F5B0916C00B395B0936C00B091CE004A
:1015900009E1BA9559F002E3BA9541F00DE7BA9521
:1015A00029F00AEFBA9511F020926C00B0916C000E
:1015B000B017A0F0B0916C00BA95B0936C00B4EB8A
:1015C000B0936B00B091CD00B093AF00F89451D8B8
:1015D0007894B091CC00B093AF0035D830D8B091AA
:1015E0006800BB2319F485FF01C08CCE01E085FDA6
:1015F00001C006E0B0919700B01708F4BBCFB091DE
:10160000BC00B35009F01FD8B0916800BB2309F4A7
:1016100079CEF8945FDD20926100209262002092E2
:101620006300522C209264002092A3007894B09121
:10163000B900BB0FB093A00020927F0020928000E1
:101640002092810020928200209283002092AC00A0
:1016500060E070E020927100B8E0B093AC00786078
:10166000EAD7B7E073FDB6E0B06CB7B9B6B1B06811
:10167000B064B6B9B6B1B6FDFDCF04B115B1B6B11F
:10168000BF77B6B9112309F00FEF0093AD0065D90C
:10169000B8E0B093AC0078608090BB00B2E0B0934B
:1016A000BB0066DD8092BB00F894BFEFB0939C0056
:1016B0009DD9B0916100B0939C00B0939D00B09310
:1016C0009E007894B1E0B0936100B09363005B2E0C
:1016D000B0936400B093A600B0919B00B093A500B6
:1016E000B091BC00B33019F49F7D87FD90627160AA
:1016F000726020926D009BDCACDC91D996D98FD9B9
:1017000094D98DD906C0F89433DD78942092AC003A
:10171000777F02DB25D8B6DBE6DB87D9F6DA66FD14
:1017200020D876FFD8D876FD06D9ACDBEEDB7DD9A4
:10173000F3DA66FD38D8A6DB28DC77D9E6DA66FD71
:101740006CD8A0DB34DC71D9E7DA66FD96D89ADB79
:101750006EDC6BD9DADAB7E073FDB6E0B06CB7B91E
:10176000B6B1B068B064B6B98DDB73DC5ED9F5D8BC
:1017700071FF23C067FD21C0B0919F00B0939C0012
:10178000B0939D00B0919B00B093A500B1E0B093E1
:10179000A60018E12CE0B0916D00B11740F07D7FFC
:1017A000746020936F00BFEFB0939C0006C0B091AF
:1017B0009700B13008F0ADCF5AC072FF10C067FD7E
:1017C0000EC0B0916F00BA9511F47B7F9CCFB0939F
:1017D0006F00B0919700B13008F09BCF48C02092C5
:1017E0007000B0919A0002E8B01708F040C085FF81
:1017F00004C0B0916800BB23D1F1B091BC00B330FC
:1018000081F495FD03C087FD04C00BC087FF01C0B4
:1018100008C067FD06C06068B0919F00B0939C004F
:101820008DCF00EF67FF05C0B0919F00B0939C0083
:1018300000E2B0917B00B01708F46BCF67FF17C0D0
:101840006F779F7D87FD90627460B2E1B0936F0007
:10185000B0919F00B0939C005CCFB0917000B395A5
:10186000B0937000B0919700BB2309F002C02092A2
:101870007000F8942FDC8090BB00B2E0B093BB0006
:1018800077DC8092BB00209261002092620020925F
:101890006300522C209264002092A0007E7F7894F6
:1018A000CAD618DCB7E0B06CB7B9B6B1B460B068EE
:1018B000B6B985FF05C0B0917000B53008F022CDF3
:1018C00055CEEDE0F0E023D00A3509F01BC0EEE084
:1018D000F0E01DD0053A09F015C03AE0A4EBB0E005
:1018E000E3E0F0E014D00D9331963A95D9F738E162
:1018F000A0ECB0E0EFE0F0E00AD00D9331963A951D
:10190000D9F702C0F4DB0AD0E7E2F0E00895E199EC
:10191000FECFEEBBFFBBE09A0DB308951ED03AE0B8
:10192000A4EBB0E0E3E0F0E00D910FD031963A95F2
:10193000D9F738E1A0ECB0E0EFE0F0E00D9105D090
:1019400031963A95D9F712D00895E199FECF0DBBA3
:10195000EEBBFFBBE29AE19A0895EDE0F0E00FEFF5
:10196000F4DFEEE0F0E00FEFF0DF0895EDE0F0E0FF
:101970000AE5EBDFEEE0F0E005EAE7DF08953091FD
:10198000B0000091B100313011F40093B800323052
:1019900011F40093B900333011F40093BA003430DD
:1019A00011F40093C600353011F40093BB003630BB
:1019B00011F40093D700373011F40093D000383081
:1019C00011F40093BC00393011F40093BD00089568
:1019D00025E03BD62A95E9F7089542D644D646D667
:1019E00048D62DD63DD63FD641D643D628D638D672
:1019F0003AD63CD63ED608953CD638D634D630D6E4
:101A00001ED637D633D62FD62BD619D632D62ED6CB
:101A10002AD626D608958090B0009090B10020D6A6
:101A20001FD61ED60CD68A94D1F723D608D69A9400
:101A3000E1F70895F894D1DF7894CADFC9DFB1E007
:101A4000B093B000B1E0B093B1002092B200F8942E
:101A5000E2DF7894B5E06B2E70909700F6D5B091E8
:101A600097007B16C9F7B13018F0BF3F40F107C0AF
:101A700086DFF89453DFB1DFB8E0B1BDA9DF6A9427
:101A800059F7B091B200B395B093B200B33008F4F7
:101A9000DECF9EDFB091B100B395B093B100F89462
:101AA000B091B000BA95EEE3F0E0EB0FF21D0491B7
:101AB00078940395B091B100B01708F4C6CF88DFD1
:101AC00087DFB091B000B395B093B000B091B00093
:101AD000BA3008F4B7CF0BDBF89420DFB8E0B1BD23
:041AE00077DFC5CB1C
:00000001FF
